:100000000C94741E189518951895189518951895B0
:100010001895189518951895189518950C94E31B34
:100020001895189518951895189518951895189568
:1000300018951895189518950C943C1B18951895BB
:1000400018951895189518950C94BF1A1895189529
:100050000C94061B189518951895189518951895D1
:0F0060000C94521918951895322E362E302E32D8
:100070000100760D0B00EA0CF60C000D0A0D140DB4
:100080001E0D280D320D3C0D460D500D0100770E52
:100090000A00BB0DDA0DEC0DFE0D100E220E340E13
:1000A000460E580E6A0E0100371008000F1014108B
:1000B00019101E10231028102D1032100100D91015
:1000C0000800A910AF10B510BB10C110C710CD109B
:1000D000D31000011C17FD16210517010717010990
:1000E00017030D17010B17090F1701121702151728
:1000F0002D1817011A171FFF16010117010317FB0F
:100100000001ED162C17015218018C1801C41801BA
:10011000EE1801FA18011219010619011E19014DF4
:1001200018022A1901FB17012018253619013D195B
:10013000014419014B19FB000001ED16ED160132C7
:1001400017013517013817013B17013E17014117F9
:10015000014417014717014A17014D1701501701B4
:100160005317015917015C17015617015F170162F8
:1001700017016517016817016B17016E17017117D9
:10018000017417017717017A17017D170180170194
:100190008317018617018917018C17018F170192A8
:1001A00017019B17019E1701A11701A417019517AD
:1001B00001981701A71701AA1701AD1701B9170177
:1001C000BC1701BF1701C21701C51701C81701B637
:1001D0001733CB1701CE1701D11701D41701D71749
:1001E00001DA1701DD1701E01701E31701E6170136
:1001F000E91701EC1701EF1701F21701F51701F8E4
:1002000017FB0001E219DA1960681908DA1908DA2F
:100210001908DA1908781908DA1908DA1908DA1940
:10022000089619089F1910BB1908D11908DA193056
:10023000DA19FB00ECEBF3E04081518162817381BC
:100240004F7F5F7F6F7F707010E00801222433249E
:10025000302C222411240024402951296229732999
:10026000ECEBF3E04083518362837383ECEBF3E0C8
:1002700010811061108310E01093C10310E01093FF
:10028000C20308950E94F41E80E090E08F3000E0E9
:1002900090073CF400E0FC01E653FC4F008301961C
:1002A000F5CF29ED33E004EF14E00E94561CA02F97
:1002B000B0E00A2F0B2B11F400E03DC0139680E054
:1002C00090E08F3000E0900738F400E0FC01E65346
:1002D000FC4F00830196F5CF2091290730912A0722
:1002E00004EF14E0201B310B2A1B3B0B2250304043
:1002F0004091290750912A0704EF14E0401B510B4D
:10030000A417B50714F000E016C040E050E0C901A2
:1003100001974817590774F48D01040F151FF80150
:10032000EC50FB4F0081FA01E653FC4F00834F5F16
:100330005F4FEDCF01E0E4E00C94FD1E0E94F51E3E
:10034000302F432F405039F04A9509F401C14A95A6
:1003500009F47DC115C241E44093F40444E540939F
:10036000F5044BE24093F60443E44093F70443E57D
:100370004093F80444E54093F90444E54093FA04BB
:100380004DE34093FB0442E24093FC0449E050E01B
:100390004093C5035093C60340E050E0483160E00D
:1003A0005607E4F5FA01E55DFB4F6081FA01E35081
:1003B000FB4F6083E5ECF3E0608171816F5F7F4FFD
:1003C00060837183FA01E350FB4F6081662319F566
:1003D00062E2FA01E350FB4F60836CE2FA01E25003
:1003E000FB4F6083E5ECF3E0608171816F5F7F4FCD
:1003F0006083718362E2FA01E150FB4F6083E5ECB8
:10040000F3E0608171816F5F7F4F60837183445F30
:100410005F4F8A0103C04F5F5F4FC0CF40E050E0A5
:10042000483160E056070CF04CC0FA01ED5BFB4F21
:100430000080B801640F751FFB01EC50FB4F008278
:10044000E5ECF3E0608171816F5F7F4F60837183C2
:10045000B801640F751FFB01EC50FB4F60816623F0
:1004600069F5A2E2B801640F751FFB01EC50FB4F68
:10047000A083ACE2B801640F751FFB01EB50FB4F8A
:10048000A083E5ECF3E0608171816F5F7F4F608353
:100490007183A2E2B801640F751FFB01EA50FB4FA4
:1004A000A083E5ECF3E0608171816F5F7F4F608333
:1004B00071834D5F5F4F040F151F03C04F5F5F4F88
:1004C000AFCF60E070E0683140E074070CF05EC1CF
:1004D000FB01E55AFB4F0080A801460F571FFA01A8
:1004E000EC50FB4F0082E5ECF3E0408151814F5F1F
:1004F0005F4F40835183A801460F571FFA01EC500C
:10050000FB4F4081442309F5A2E2A801460F571F83
:10051000FA01EC50FB4FA083ADE0A801460F571F36
:10052000FA01EB50FB4FA083E5ECF3E040815181F1
:100530004F5F5F4F40835183A0E0A801460F571FD4
:10054000FA01EA50FB4FA08321C16F5F7F4FBBCF01
:1005500041E44093F40444E54093F5044BE24093B6
:10056000F60443E44093F70444E44093F8044EE473
:100570004093F90443E54093FA0447E44093FB04B5
:1005800049E44093FC0440E54093FD044DE340936F
:10059000FE0442E24093FF044CE050E04093C50368
:1005A0005093C60320E040E050E0483460E0560736
:1005B00094F5FA01E752FC4F6081FA01E050FB4FDD
:1005C0006083E5ECF3E0608171816F5F7F4F608352
:1005D0007183FA01E050FB4F60816623C9F462E247
:1005E000FA01E050FB4F60836DE0FA01EF5FFA4FD4
:1005F0006083E5ECF3E0608171816F5F7F4F608322
:10060000718360E0FA01EE5FFA4F608321E003C07E
:100610004F5F5F4FCACF2223C9F442E2409348059F
:10062000E5ECF3E0408151814F5F5F4F40835183A0
:100630004DE040934905E5ECF3E0408151814F5F87
:100640005F4F4083518340E040934A059FC041E49F
:100650004093F40444E54093F5044BE24093F604E0
:1006600043E44093F70449E44093F80440E54093A1
:10067000F90443E54093FA0444E54093FB0441E464
:100680004093FC0442E54093FD0444E54093FE049E
:100690004DE34093FF0442E24093000544E540935C
:1006A000010543E44093020540E54093030542E21F
:1006B000409304054CE24093050542E24093060551
:1006C00080E090E040E050E0483460E0560794F469
:1006D000CA01FC01E653FC4F6081662359F0FC011E
:1006E000E653FC4F6081FC01E95FFA4F60834F5F86
:1006F0005F4FEACF42E2FC01E95FFA4F4083019687
:100700004CE2FC01E95FFA4F4083019620E040E0B3
:1007100050E0453060E05607FCF4FA01EF5DFB4F16
:100720006081FC01E95FFA4F6083FC01E95FFA4FE9
:100730006081662369F44DE0FC01E95FFA4F408374
:10074000019640E0FC01E95FFA4F408321E004C0DC
:1007500001964F5F5F4FDDCF222359F44DE0FC013E
:10076000E95FFA4F4083019640E0FC01E95FFA4FF0
:100770004083FC017396E093C503F093C60306C063
:1007800040E050E04093C5035093C603E3E00C946F
:10079000FE1E0E94F41ED801C9018C010E943D1C5E
:1007A0000093C5031093C6030091C5031091C603BF
:1007B000063222E0120730F006E212E00093C50391
:1007C0001093C60300E010E02091C5033091C603EA
:1007D0000217130748F4FC012081FD0120831196C4
:1007E00001960F5F1F4FF0CFE4E00C94FD1E20E454
:1007F00031E004EF14E0CDDFE7E2F7E00081077FAE
:10080000008301E00093C10302E00093C203089556
:100810002FE431E004EF14E00E94461C002319F499
:1008200007E008DD089522E531E004EF14E00E94BE
:10083000461C002341F0ECEBF3E0008108600083EC
:1008400000E0F8DC089524E631E004EF14E00E94B3
:10085000461C002309F043C026E731E004EF14E012
:100860000E94461C0023D9F526E831E004EF14E08D
:100870000E94461C002399F527E931E004EF14E0BB
:100880000E94461C002359F529EA31E004EF14E0E8
:100890000E94461C002319F52AEB31E004EF14E016
:1008A0000E94461C0023D9F420ED31E004EF14E04F
:1008B0000E94461C002399F423EE31E004EF14E07B
:1008C0000E94461C002359F425EF31E004EF14E0A8
:1008D0000E94461C002319F408E0ACDC089503E0F4
:1008E0000093C203089526E032E004EF14E051DFE4
:1008F000E7E2F7E00081077F008301E00093C10396
:1009000004E00093C20300E010E000937D04109324
:100910007E040895EDE7F4E0008111810F5F1F4F21
:100920000083118323E132E004EF14E00E94461CAF
:100930000023D1F4E0917D04F0917E04F89718F043
:1009400009E078DC0895E7E2F7E0008102600083C7
:10095000E7E2F7E00081077F008302E00093C10334
:1009600004E00093C203089505E00093C2030895D4
:1009700020E431E004EF14E00CDFE7E2F7E000816F
:10098000077F008301E00093C10306E00093C203E8
:1009900008952FE431E004EF14E00E94461C002388
:1009A00019F40CE047DC089524E631E004EF14E08C
:1009B0000E94461C002309F04FC022E531E004EFFD
:1009C00014E00E94461C002309F043C026E731E0F2
:1009D00004EF14E00E94461C0023D9F526E831E01C
:1009E00004EF14E00E94461C002399F527E931E04A
:1009F00004EF14E00E94461C002359F529EA31E077
:100A000004EF14E00E94461C002319F52AEB31E0A4
:100A100004EF14E00E94461C0023D9F420ED31E0DD
:100A200004EF14E00E94461C002399F423EE31E009
:100A300004EF14E00E94461C002359F425EF31E036
:100A400004EF14E00E94461C002319F40AE0F2DBD4
:100A500008950BE0EFDB089507E00093C2030895CB
:100A60002BE132E004EF14E094DEE7E2F7E00081EE
:100A7000077F008301E00093C10308E00093C203F5
:100A800008952FE431E004EF14E00E94461C002397
:100A900019F40DE0CFDB089509E00093C203089537
:100AA00000E04CDCE7E2F7E00081077F008301E033
:100AB0000093C1030AE00093C20308952FE431E0DC
:100AC00004EF14E00E94461C002319F40EE0B2DB90
:100AD00008950BE00093C203089529E232E004EF89
:100AE00014E057DEE7E2F7E00081077F008301E0D2
:100AF0000093C1030CE00093C20300E00093C7031E
:100B000008950091C70303950093C7032FE431E0D4
:100B100004EF14E00E94461C0023C1F40091C703B7
:100B20000C3418F00FE086DB0895E7E2F7E000816F
:100B300002600083E7E2F7E00081077F008302E0C4
:100B40000093C1030CE00093C203089520E431E058
:100B500004EF14E01EDEE7E2F7E00081077F008388
:100B600001E00093C1030FE00093C203089527E959
:100B700031E004EF14E00E94461C002319F401E167
:100B800059DB08950DE00093C203089524E332E099
:100B900004EF14E0FEDDE7E2F7E00081077F008369
:100BA00001E00093C1030EE00093C203089500E149
:100BB0000093C203089520E431E004EF14E0E9DD7E
:100BC000E7E2F7E00081077F008301E00093C103C3
:100BD00001E10093C20308952FE431E004EF14E033
:100BE0000E94461C002319F409E124DB089529EA38
:100BF00031E004EF14E00E94461C002309F04FC0CE
:100C000022E531E004EF14E00E94461C002309F0C5
:100C100043C026E731E004EF14E00E94461C0023A5
:100C2000D9F526E831E004EF14E00E94461C0023C9
:100C300099F527E931E004EF14E00E94461C0023F7
:100C400059F524E631E004EF14E00E94461C00232D
:100C500019F52AEB31E004EF14E00E94461C002352
:100C6000D9F420ED31E004EF14E00E94461C00238B
:100C700099F423EE31E004EF14E00E94461C0023B7
:100C800059F425EF31E004EF14E00E94461C0023E4
:100C900019F40BE1CFDA08950AE1CCDA08950E9445
:100CA0005B1E002321F005E10093C20303C002E1B3
:100CB0000093C20300E010E000937D0410937E04D3
:100CC000089501E03BDBE7E2F7E00081077F008366
:100CD00001E00093C10303E10093C20308952FE4F0
:100CE00031E004EF14E00E94461C002359F42FE386
:100CF00032E004EF14E00E94461C002319F006E1E4
:100D000099DA089504E10093C20308958A93BADA48
:100D1000802F882319F407E18DDA03C005E10093E1
:100D2000C2038991089502E009DBE7E2F7E0008160
:100D3000077F008301E00093C10306E10093C20333
:100D40000895EDE7F4E0008111810F5F1F4F0083EC
:100D5000118328E432E004EF14E00E94461C0023D3
:100D600041F020E532E004EF14E00E94461C00232D
:100D700011F100917D0410917E04063920E01207E4
:100D800049F408E157DA00E010E000937D04109385
:100D90007E040895E7E2F7E0008102600083E7E265
:100DA000F7E00081077F008302E00093C10306E1C2
:100DB0000093C203089507E10093C20300E010E02E
:100DC00000937D0410937E040895ECEBF3E0008122
:100DD0000860008300E02EDA089520E431E004EF9B
:100DE00014E0D7DCECEBF3E00081077F0083E7E25F
:100DF000F7E00081077F008301E00093C10309E170
:100E00000093C20308952FE431E004EF14E00E9440
:100E1000461C002319F40CE10DDA089524E631E0B4
:100E200004EF14E00E94461C002341F423EE31E05D
:100E300004EF14E00E94461C002341F0ECEBF3E0C9
:100E40000081077F008300E0F5D9089522E531E0B5
:100E500004EF14E00E94461C0023D9F526E731E098
:100E600004EF14E00E94461C002399F526E831E0C7
:100E700004EF14E00E94461C002359F527E931E0F5
:100E800004EF14E00E94461C002319F529EA31E022
:100E900004EF14E00E94461C0023D9F42AEB31E051
:100EA00004EF14E00E94461C002399F420ED31E089
:100EB00004EF14E00E94461C002359F425EF31E0B2
:100EC00004EF14E00E94461C002319F40DE1B2D98E
:100ED00008950AE10093C203089525E532E004EF86
:100EE00014E057DCE7E2F7E00081077F008301E0D0
:100EF0000093C1030BE10093C203089500E09AD967
:100F0000089526E032E004EF14E043DCE7E2F7E086
:100F10000081077F008301E00093C1030DE100938E
:100F2000C20308950EE10093C203089520E431E066
:100F300004EF14E02EDCE7E2F7E00081077F008396
:100F400001E00093C1030FE10093C20308952FE471
:100F500031E004EF14E00E94461C002319F400E283
:100F600069D9089524E631E004EF14E00E94461C9C
:100F7000002341F0ECEBF3E00081077F008300E009
:100F800059D9089525E632E004EF14E00E94461C8A
:100F9000002309F043C026E731E004EF14E00E948B
:100FA000461C0023D9F526E831E004EF14E00E9446
:100FB000461C002399F527E931E004EF14E00E9474
:100FC000461C002359F529EA31E004EF14E00E94A1
:100FD000461C002319F52AEB31E004EF14E00E94CF
:100FE000461C0023D9F420ED31E004EF14E00E9408
:100FF000461C002399F423EE31E004EF14E00E9434
:10100000461C002359F425EF31E004EF14E00E9460
:10101000461C002319F401E20DD9089502E20AD911
:1010200008952AE732E00FE714E00E94951C009132
:101030007304109174040E94AB1C24E337E00FE7A3
:1010400014E00E94A01C27E832E00FE714E00E94A1
:10105000A01C0FE714E00E943D1C0093C5031093F1
:10106000C603E7E2F7E00081077F00830CE000930E
:10107000C10301E20093C20308952AE832E00FE7BA
:1010800014E00E94461C002319F003E2D3D808950F
:1010900025E932E00FE714E00E94461C002319F016
:1010A00004E2C8D808952FE932E00FE714E00E9467
:1010B000461C002319F005E2BDD8089527EA32E066
:1010C0000FE714E00E94461C002351F00CE200934D
:1010D000C20300E010E000937D0410937E040895A5
:1010E00006E2A8D808950091730410917404009347
:1010F000C5031093C60309E00093C10303E2009304
:10110000C2030895E0ECF3E0008100FF04C008E0B2
:101110000093C103089500E08DD80895E7E2F7E059
:10112000008102600083E7E2F7E00081077F00832F
:1011300002E00093C10305E20093C20308952FE982
:1011400032E004EF14E00E94461C002369F000E046
:1011500010E000937D0410937E0400E00093C1032F
:1011600008E20093C2030895EDE7F4E000811181E5
:101170000F5F1F4F0083118300917D0410917E0447
:10118000093120E0120741F4ECEBF3E000810F7D20
:10119000008307E24FD80895C1DF08950AE2009363
:1011A000F40408E00093F50401E40093F6040AE077
:1011B0000093F70401E80093F80402EA0093F904AD
:1011C00001E00093FA0405E00093FB040091AC03F6
:1011D0000093FC040091AD030093FD040091AE0365
:1011E0000093FE040091AF030093FF040091B0034D
:1011F000009300050091B103009301050091B20333
:10120000009302050091B303009303050091B4031A
:10121000009304050091B503009305050091B60302
:10122000009306050091B703009307050091B803EA
:10123000009308050091B903009309050091BA03D2
:1012400000930A050091BB0300930B050091750400
:101250001091760400930C050091750410917604AA
:10126000012F10E000930D0504E100930E0500E04E
:1012700000930F0500E00093100500E000931105B6
:101280000EE110E00093C5031093C60309E000933C
:10129000C10307E20093C203089500E00E941A010F
:1012A000089529EA32E004EF14E073DAE7E2F7E0A8
:1012B0000081077F008301E00093C10309E20093EE
:1012C000C2030895E7E2F7E0008102600083E7E2ED
:1012D000F7E00081077F008302E00093C10309E289
:1012E0000093C20308959A938A9380E090E02CEBD8
:1012F00032E004EF14E00E94461C002309F45FC0B2
:101300002091290730912A0704EF14E0201B04EFF5
:1013100014E00E94131DC801082F092B01F5EDE709
:10132000F4E0008111810F5F1F4F00831183009152
:101330007D0410917E04083A21E6120749F4ECEB93
:10134000F3E000810F7D008309E20E941A016AC068
:1013500000E00093C10308E20093C20363C08E3132
:1013600000E0900749F0ECEBF3E000810F7D008393
:101370000AE20E941A0156C0ECEBF3E00081006221
:1013800000832091290730912A0704EF14E0201BE5
:10139000310B04EF14E00E949D1D0093790410931B
:1013A0007A040091790410917A04012B21F406E368
:1013B0000E941A0137C000E00E941A0133C0209138
:1013C000290730912A0704EF14E0201B310BD9F4D0
:1013D000E8ECF3E0008111810F5F1F4F0083118360
:1013E0000091C8031091C903003325E7120721F4C7
:1013F00008E20E941A0116C000E00093C1030EE249
:101400000093C2030FC02AEC32E004EF14E00E9404
:10141000461C002321F00EE20E941A0103C00FE2D5
:101420000E941A018991999108950091790410916F
:101430007A04012B09F448C00091790410917A04D0
:10144000073222E0120738F006E212E00093770438
:101450001093780408C00091790410917A040093E5
:1014600077041093780420ED32E004EF14E00E943A
:10147000951C00917704109178040E94AB1C24E322
:1014800037E004EF14E00E94A01C27E832E004EFEC
:1014900014E00E94A01C04EF14E00E943D1C009385
:1014A000C5031093C603E7E2F7E00081077F0083DE
:1014B00001E00093C103ECEBF3E0008100620083E4
:1014C0000BE20093C2030895ECEBF3E000810F7D83
:1014D000008300E00E941A0108959A938A932CEBEE
:1014E00032E004EF14E00E94461C002309F46CC0B3
:1014F0002091290730912A0704EF14E0201B04EF04
:1015000014E00E94131D00937B0410937C0400914F
:101510007B0410917C04012B21F401E30E941A0149
:1015200086C00091790410917A0420917B04309157
:101530007C040217130778F400E010E000937904AC
:1015400010937A04ECEBF3E000810F7D008302E35B
:101550000E941A016CC02091290730912A0704EFDC
:1015600014E0201B310B04EF14E00E94391EC80167
:1015700020E030E000917B0410917C0420173107BB
:1015800070F48901080F191FF801EC50FB4F00811E
:10159000F901EC50FB4F00832F5F3F4FEBCF0091E1
:1015A0007B0410917C04E9E7F4E020813181201B69
:1015B000310B20833183ECEBF3E000810062008388
:1015C00000E00E941A0133C02091290730912A07B8
:1015D00004EF14E0201B310BD9F4E8ECF3E00081B8
:1015E00011810F5F1F4F008311830091C803109179
:1015F000C903003325E7120721F403E30E941A010F
:1016000016C000E00093C10301E30093C2030FC0C2
:101610002AEC32E004EF14E00E94461C002321F083
:1016200004E30E941A0103C005E30E941A01899194
:10163000999108950AE20093F40408E00093F504F8
:1016400001E40093F6040AE00093F70401E8009334
:10165000F80402EA0093F90401E00093FA0405E0BB
:101660000093FB040091AC030093FC040091AD03D4
:101670000093FD040091AE030093FE040091AF03BC
:101680000093FF040091B003009300050091B103A3
:10169000009301050091B203009302050091B3038A
:1016A000009303050091B403009304050091B50372
:1016B000009305050091B603009306050091B7035A
:1016C000009307050091B803009308050091B90342
:1016D000009309050091BA0300930A050091BB032A
:1016E00000930B05009175041091760400930C058E
:1016F0000091750410917604012F10E000930D0500
:1017000004E100930E0500E000930F0500E0009354
:10171000100500E0009311050EE110E00093730442
:10172000109374040895E7E2F7E00081077F0083D7
:1017300000917304109174040093C5031093C603C1
:1017400001E00093C1030DE20093C2030895E7E2B4
:10175000F7E0008102600083E7E2F7E00081077FA5
:10176000008302E00093C1030DE20093C2030895D9
:101770002FE932E004EF14E00E94461C002331F10F
:10178000E0ECF3E0008100FF18C0ECEBF3E0018136
:101790000260018300E010E000937D0410937E045A
:1017A00000E010E00093C8031093C90300E0009329
:1017B000C10308E20093C2030895ECEBF3E001815A
:1017C0000160018300E00E941A010895EDE7F4E052
:1017D000008111810F5F1F4F0083118300917D04F1
:1017E00010917E04093120E0120721F40DE20E94DD
:1017F0001A010895ACDF089520EE32E004EF14E002
:101800000E94C903E7E2F7E00081077F008301E05F
:101810000093C10300E30093C20308952FE431E075
:1018200004EF14E00E94461C002321F400E30E9410
:101830001A01089501E00093C203089505E600939C
:10184000C20300E00093C303089520EF32E004EFE9
:1018500014E00E94C903E7E2F7E00081077F0083FC
:1018600001E00093C10301E70093C20308952FE450
:1018700031E004EF14E00E94461C002321F403E44D
:101880000E941A01089500E00E941A010895289A02
:1018900006E60093C20300EB14E00093910410935A
:1018A000920401E00093C3030895E8E2F7E00081A9
:1018B0000D7F008300919104109192040E94381CC6
:1018C000E8E2F7E00081016000830E94081A01E06D
:1018D0000E94181A07E60093C2030895E8E2F7E0B1
:1018E000008100FF04C007E60093C203089508E6E4
:1018F0000093C20308950091C303015029F00A9593
:1019000039F00A95B9F01FC009E60093C2030895A3
:10191000E0ECF3E0008102FF09C0E0ECF3E00081BD
:101920000B7F008304E60093C20308950AE6009348
:10193000C2030895ECEBF3E00081016000830BE645
:101940000093C2030895ECEBF3E000811181228142
:1019500033810F7F1F7F2F7F307000601060206009
:101960003464ECEBF3E0008311832283338300E0E3
:101970000093C2030895289806E60093C20304EC7E
:1019800019E0009391041093920402E00093C303C2
:10199000089508EB1BE0009391041093920403E078
:1019A0000093C30306E60093C20308950CE6009378
:1019B000C203089500E00093930401E00093C40380
:1019C0000DE60093C20308950091C403E0E7F0E040
:1019D0000C94AB1E0E94390F26EF32E004EF14E0A6
:1019E0000E94C9030EE60093C20308952BEF32E074
:1019F00004EF14E00E94C9030EE60093C2030895A9
:101A000028E033E004EF14E00E94C9030EE60093DF
:101A1000C203089524E133E004EF14E00E94C903F7
:101A20000EE60093C203089520E233E004EF14E0D1
:101A30000E94C9030EE60093C203089526E233E034
:101A400004EF14E00E94C9030EE60093C203089558
:101A50002CE233E004EF14E00E94C9030EE6009389
:101A6000C203089522E333E004EF14E00E94C903A7
:101A70000EE60093C20308952DE333E004EF14E073
:101A80000E94C9030EE60093C20308952CE433E0DC
:101A900004EF14E00E94C9030EE60093C203089508
:101AA000ECEBF3E000811181228133810F7F1F7FF6
:101AB0002F7F30700083118322833383ECEBF3E0BC
:101AC000008100610083ECEBF3E000810F7B008379
:101AD000ECEBF3E000810260008300E00093C403BC
:101AE00000E00093C10300E00093C2030895E7E221
:101AF000F7E00081077F008301E00093C1030FE658
:101B00000093C2030895ECEBF3E0408151816281C0
:101B100073814F7F5F7F6F7F707010E00801222418
:101B20003324302C222411240024402951296229F5
:101B30007329ECEBF3E04083518362837383ECEB16
:101B4000F3E0108110611083ECEBF3E010811F7B58
:101B50001083ECEBF3E010811D7F108310E01093F5
:101B6000C10310E01093C20308950091C403ECE890
:101B7000F0E00C94AB1E0091930403950093930442
:101B80002FE431E004EF14E00E94461C002359F4D6
:101B900000919304053019F40AE3B5DF08950DE6CA
:101BA0000093C203089502E00093C4030DE600937E
:101BB000C20308952FE431E004EF14E00E94461CB4
:101BC000002319F40BE39FDF089503E00093C4039F
:101BD0000DE60093C20308952FE431E004EF14E012
:101BE0000E94461C002319F40CE38DDF089504E0E5
:101BF0000093C4030DE60093C20308952FE431E07F
:101C000004EF14E00E94461C002319F40DE37BDF6F
:101C1000089505E00093C4030DE60093C203089500
:101C20002FE431E004EF14E00E94461C002319F475
:101C30000EE369DF089506E00093C4030DE6009308
:101C4000C20308952FE431E004EF14E00E94461C23
:101C5000002319F40FE357DF089507E00093C4034E
:101C60000DE60093C20308952FE431E004EF14E081
:101C70000E94461C002319F400E445DF089508E0A3
:101C80000093C4030DE60093C20308952FE431E0EE
:101C900004EF14E00E94461C002319F401E433DF32
:101CA000089509E00093C4030DE60093C20308956C
:101CB0002FE431E004EF14E00E94461C002319F4E5
:101CC00002E421DF08950AE00093C4030DE60093C7
:101CD000C20308950E947B11002319F400E513DF6D
:101CE00008950BE00093C4030DE60093C20308952A
:101CF00020E431E004EF14E00E94C903E7E2F7E0DA
:101D00000081077F008301E00093C10303E7009394
:101D1000C20308952FE431E004EF14E00E94461C52
:101D2000002321F405E40E941A01089528E432E01A
:101D300004EF14E00E94461C002359F14091730403
:101D40005091740428EA34E004EF14E00E94EF1C80
:101D50000091730410917404E5E7F4E0208131816F
:101D6000201B310B20833183009175041091760480
:101D7000012B31F4E0ECF3E000810160008305C049
:101D8000E0ECF3E000810E7F008300E20093C203E9
:101D9000089524E533E004EF14E00E94461C00237C
:101DA00021F006E40E941A0108952CE533E004EFC7
:101DB00014E00E94461C002321F007E40E941A014F
:101DC000089522E633E004EF14E00E94461C00234D
:101DD00021F008E40E941A01089529E633E004EF97
:101DE00014E00E94461C002321F009E40E941A011D
:101DF000089521E733E004EF14E00E94461C00231D
:101E000021F00AE40E941A01089528E733E004EF64
:101E100014E00E94461C002321F00BE40E941A01EA
:101E2000089523E833E004EF14E00E94461C0023E9
:101E300021F00CE40E941A0108952BE833E004EF2E
:101E400014E00E94461C002321F00DE40E941A01B8
:101E5000089522E933E004EF14E00E94461C0023B9
:101E600021F00EE40E941A0108950FE40E941A0165
:101E7000089502E015B1102715B908950FEF04B9C0
:101E800002E005B90FEF07B900E008B90FEF0AB992
:101E900000E00BB9089500916000086100936000B4
:101EA00008E200936000009160000064009360000D
:101EB00008951C0108010FEF1FEF41E250E181E09E
:101EC00090E082179307D4F4F001E80FF91F7081B6
:101ED00060E006271727E0E0F0E0E83060E0F60772
:101EE0005CF417FB2EF4000F111F0427152702C006
:101EF000000F111F3196F1CF0196E3CFC101089574
:101F00000E94F41E00911F0710912007F801ED5563
:101F1000FB4FB081A0E000911F0710912007F8014E
:101F2000EE55FB4F008110E0A00FB11F80911F07FD
:101F30009091200702979C0104EA14E0BADF98010F
:101F40002A173B0711F000E002C00091A704E4E06B
:101F50000C94FD1E0E94FC19EDE1F7E0008101FDEB
:101F600002C0A895F9CF0895302F132F105029F0F3
:101F70001A9529F11A95E9F13EC0ECEBF3E01081D6
:101F80001170ECEBF3E0208121FB20E021F9122B12
:101F9000ECEBF3E0208123FB20E023F9122BECEBA8
:101FA000F3E0208124FB20E024F9122BECEBF3E09A
:101FB000208125FB20E025F9122B012F0895ECEB61
:101FC000F3E0118111701170ECEBF3E0218121FB42
:101FD00020E020F92170220F122BECEBF3E021819D
:101FE00022FB20E020F92170220F220F122B012F5B
:101FF000089500E0089500E008950E94F01EF09119
:10200000A604E0E00091A50410E0E00FF11F339773
:102010003F010091A804E6EAF0E00C94AB1E8FE0CB
:102020000AEC13E0280124C085E001E214E0280155
:102030001FC088E409ED13E028011AC085E006E21C
:1020400014E0280115C088E10BE214E0280110C05B
:1020500088E103E414E028010BC088E10BE514E0FB
:10206000280106C080E10CEA13E0280101C080E0ED
:10207000082F10E00615170510F497E336C090E01E
:1020800000E010E0282F30E00217130754F420E09E
:10209000F201208321E0420E20E0521E0F5F1F4F0D
:1020A000F1CF082F10E0119501951040400E511E00
:1020B00000E010E00615170568F4F801EC55FB4F39
:1020C0002681F201208321E0420E20E0521E0F5FA4
:1020D0001F4FF0CFE7E2F7E00081077F008300E0C9
:1020E0000093C10300E00093C20304E00093A40442
:1020F00001E00093A50400E00093A604ECEBF3E0FC
:10210000008104FF03C09093A70403C001E3009380
:10211000A70424E030E004EA14E0CBDED8010A2F63
:102120000093A8048D01012F10E00093A90406E09C
:1021300010E000932107109322070CDFE8E00C94D5
:10214000F91E0E94F01E0091A804ECEBF0E00C9444
:10215000AB1E0FE0602E0AEC13E0D8012BC005E0A7
:10216000602E01E214E0D80125C008E4602E09EDDC
:1021700013E0D8011FC005E0602E06E214E0D8018C
:1021800019C008E1602E0BE214E0D80113C008E189
:10219000602E03E414E0D8010DC008E1602E0BE5C9
:1021A00014E0D80107C000E1602E0CEA13E0D8016A
:1021B00001C06624662019F408E3702E1FC077243E
:1021C00080E090E000E010E0262D30E002171307D9
:1021D00054F42C91F801EC55FB4F24831196019691
:1021E0000F5F1F4FF1CFE7E2F7E00081077F008329
:1021F00000E00093C10300E00093C20304E00093F9
:10220000A404082F03950093A504FC013196EF2F39
:10221000F0E0E093A604ECEBF3E0008104FF03C0E0
:102220007092A70403C001E30093A7049C012C5FF4
:102230003F4F04EA14E03DDE2801042DFC01EC557B
:10224000FB4F04838201012F10E0FC01EC55FB4F92
:102250000583FC013696E0932107F09322077ADE8E
:10226000E8E00C94F91E9A938A9304E00093A40486
:1022700008E10093A50400E00093A60400E00093A9
:10228000A70400E010E0073020E012075CF4F8013A
:10229000E859FF4F2491F801EC55FB4F24830F5F61
:1022A0001F4FF1CF00E010E0003120E012075CF496
:1022B000F801EC56FB4F2081F801EC55FB4F2387CA
:1022C0000F5F1F4FF1CF2BE130E004EA14E0F1DDA6
:1022D000C801082F0093BF048C01012F10E0009368
:1022E000C0040DE110E0009321071093220732DEB5
:1022F0008991999108950E94F21E28E933E004EF34
:1023000014E00E94461C002341F02BE933E004EF67
:1023100014E00E94461C002311F400E064C08FEF1B
:102320009FEF00E010E04091290750912A0724EF29
:1023300034E0421B530B041715076CF4F801EC5002
:10234000FB4F20812A3321F40F5F1F4FC80103C0C8
:102350000F5F1F4FE8CF8F3F0FEF900711F400E0A2
:1023600042C0AFEFBFEF8C014091290750912A077F
:1023700024EF34E0421B530B041715079CF4F801BB
:10238000EC50FB4F20812D3051F4F801EB50FB4F06
:1023900020812A3021F401501040D80103C00F5F82
:1023A0001F4FE2CFFD01E81BF90B31962F0101E130
:1023B000401600E050061CF000E1402E552420E0BD
:1023C00030E02415350574F48C01020F131FF80159
:1023D000EC50FB4F0081F901EC56FB4F00832F5F5F
:1023E0003F4FEFCF01E0E6E00C94FB1E9A938A93F7
:1023F00004E00093A40402E00093A50400E000932D
:10240000A60405E00093A70405E00093A80425E0D6
:1024100030E004EA14E04DDDC801082F0093A90460
:102420008C01012F10E00093AA0407E010E0009354
:102430002107109322078EDD8991999108959A932F
:102440008A9304E00093A40407E00093A50400E04D
:102450000093A60400E00093A704ECEBF3E00081F6
:10246000118122813381032F10E020E030E00093BE
:10247000A80400E079DD0093A90401E075DD009374
:10248000AA0402E071DD0093AB0400E00093AC0409
:102490000091C2030093AD042AE030E004EA14E0A6
:1024A00008DDC801082F0093AE048C01012F10E055
:1024B0000093AF040CE010E0009321071093220773
:1024C00049DD8991999108959A938A9304E0009344
:1024D000A40401E00093A50400E00093A60401E039
:1024E0000093A70424E030E004EA14E0E2DCC80131
:1024F000082F0093A8048C01012F10E00093A90479
:1025000006E010E0009321071093220723DD899154
:10251000999108950E94F51EF091A604E0E00091C3
:10252000A50410E0E00FF11F3197E093C503F0938D
:10253000C6030091C5031091C603073222E01207BB
:1025400010F0A6E013C0A0E04091C5035091C6036F
:1025500028EA34E004EF14E00E94EF1CE7E2F7E021
:102560000081077F008301E00093C10304E0009332
:10257000A40401E00093A50400E00093A604ECEBA2
:10258000F3E0008104FF03C0A093A70403C001E3AC
:102590000093A70424E030E004EA14E08ADCC801D8
:1025A000082F0093A8048C01012F10E00093A904C8
:1025B00006E010E00093210710932207CBDC01E036
:1025C00000931A07ECEBF3E000810F7E0083E3E059
:1025D0000C94FE1E0E94F41E80E091E004E0009343
:1025E000A404082F03950093A504FC013196EF2F56
:1025F000F0E0E093A60400E00093A70400E010E000
:102600000817190758F4F801EC50FB4F2081F80126
:10261000EC55FB4F24830F5F1F4FF2CFFC01349624
:102620009F0104EA14E045DCD8010A2FFC01EC55B7
:10263000FB4F04838D01012F10E0FC01EC55FB4F93
:102640000583FC013696E0932107F093220782DC94
:10265000E4E00C94FD1E0E94F51E0091A804A02F3A
:1026600004E00093A40401E00093A50400E00093BB
:10267000A604ECEBF3E0008104FF04C000E000934B
:10268000A70403C001E30093A70424E030E004EAB8
:1026900014E00FDCC801082F0093A8048C01012F5F
:1026A00010E00093A90406E010E0009321071093C6
:1026B000220750DCECEBF3E00081118122813381B1
:1026C0000F7F1F7F2F7F307000831183228333831E
:1026D000ECEBF3E00081077F00830091A704002367
:1026E00051F4AA2321F004E00093C10307C005E0E0
:1026F0000093C10303C000E00093C103ECEBF3E0DF
:1027000000810F7D0083E3E00C94FE1E9A938A9370
:1027100004E00093A40401E00093A50400E000930A
:10272000A60400E00093A70424E030E004EA14E0EB
:10273000C0DBC801082F0093A8048C01012F10E012
:102740000093A90406E010E00093210710932207EC
:1027500001DCECEBF3E000811181228133810F7FFA
:102760001F7F2F7F30700083118322833383ECEB34
:10277000F3E0008100640083ECEBF3E000810F7E66
:102780000083ECEBF3E000810E7F0083E0ECF3E0EC
:1027900000810460008302E30093C1038991999151
:1027A00008959A938A9304E00093A40401E00093AF
:1027B000A50400E00093A60400E00093A70424E031
:1027C00030E004EA14E075DBC801082F0093A80488
:1027D0008C01012F10E00093A90406E010E00093A3
:1027E000210710932207B6DBECEBF3E000811181A7
:1027F000228133810F7F1F7F2F7F307000831183F1
:1028000022833383ECEBF3E000810F7E008303E34C
:102810000093C1038991999108959A938A93309175
:10282000A90420E00091A80410E0200F311F20939C
:102830007504309376040E941A0B04E00093A404FC
:1028400001E00093A50400E00093A604ECEBF3E0A4
:10285000008104FF04C000E00093A70403C001E36B
:102860000093A70424E030E004EA14E022DBC8016E
:10287000082F0093A8048C01012F10E00093A904F5
:1028800006E010E0009321071093220763DBECEBD6
:10289000F3E000811181228133810F7F1F7F2F7F21
:1028A00030700083118322833383ECEBF3E00081EB
:1028B0000F7D0083ECEBF3E001810E7F0183ECEBF5
:1028C000F3E001810D7F01830091A704002349F407
:1028D000E0ECF3E000810E7F008307E00093C1038A
:1028E00003C000E00093C1038991999108950E946B
:1028F000F41E80E0F091A604E0E00091A50410E051
:10290000E00FF11F3197E0937304F093740400918A
:10291000730410917404073222E0120710F080E370
:1029200034C00091750410917604209173043091A5
:1029300074040217130710F482E327C04091730454
:102940005091740428EA34E004EF14E00E94EF1C74
:102950000091730410917404E5E7F4E02081318163
:10296000201B310B20833183009175041091760474
:10297000012B31F4E0ECF3E000810160008305C03D
:10298000E0ECF3E000810E7F008304E00093A404F8
:1029900001E00093A50400E00093A604ECEBF3E053
:1029A000008104FF03C08093A70403C001E30093E8
:1029B000A70424E030E004EA14E00E94590FD80193
:1029C0000A2F0093A8048D01012F10E00093A904A1
:1029D00006E010E00093210710932207BBDAECEB2E
:1029E000F3E000811181228133810F7F1F7F2F7FD0
:1029F000307090E0AC0160E070E0742F60E050E077
:102A000040E0042B152B262B372BECEBF3E0008357
:102A10001183228333830091A704002349F4ECEB54
:102A2000F3E000810F7E008307E00093C10303C041
:102A300000E00093C103E4E00C94FD1E9A938A9396
:102A400004E00093A40403E00093A50400E00093D5
:102A5000A604ECEBF3E0008104FF04C000E0009367
:102A6000A70403C001E30093A70400917904109127
:102A70007A040093A8040091790410917A04012F3C
:102A800010E00093A90426E030E004EA14E00E947C
:102A9000590FC801082F0093AA048C01012F10E0E0
:102AA0000093AB0408E010E0009321071093220785
:102AB0000E94AA0FECEBF3E00081118122813381A7
:102AC0000F7F1F7F2F7F307000831183228333831A
:102AD0000091A704002321F40BE00093C10303C07D
:102AE00000E00093C1038991999108959A938A9384
:102AF000ECEBF3E000811181228133810F7F1F7F96
:102B00002F7F3070008311832283338304E000938E
:102B1000A40400917B0410917C04073222E0120788
:102B200040F101E00093A50400E00093A604ECEB63
:102B3000F3E0008104FF04C000E30093A70403C096
:102B400001E30093A70424E030E004EA14E00E94CB
:102B5000590FC801082F0093A8048C01012F10E021
:102B60000093A90406E010E00093210710932207C8
:102B70005EC000917B0410917C0403950093A50432
:102B8000E0917B04F0917C043196EF2FF0E0E0932C
:102B9000A604ECEBF3E0008104FF04C000E0009326
:102BA000A70403C001E30093A70400917B041091E4
:102BB0007C04012BA1F000E010E020917B04309117
:102BC0007C040217130758F4F801EC50FB4F2081E6
:102BD000F801EC55FB4F24830F5F1F4FEECF209180
:102BE0007B0430917C042C5F3F4F04EA14E00E9488
:102BF000590FC801082F20917B0430917C04F90102
:102C0000EC55FB4F04838C01012F10E020917B04D5
:102C100030917C04F901EC55FB4F0583E0917B0476
:102C2000F0917C043696E0932107F09322070E94EE
:102C3000AA0F00E00093C103899199910895192F7B
:102C4000282F80E090E08F3000E090073CF400E017
:102C5000FC01E653FC4F00830196F5CF80E090E045
:102C6000883400E090073CF400E0FC01E752FC4FA0
:102C700000830196F5CF80E090E0853000E090077A
:102C80003CF400E0FC01EF5DFB4F00830196F5CFC3
:102C900080E090E0853000E090073CF400E0FC012B
:102CA000EA5DFB4F00830196F5CF80E090E088312C
:102CB00000E090073CF400E0FC01E55DFB4F008381
:102CC0000196F5CF80E090E0883100E090073CF479
:102CD00000E0FC01ED5BFB4F00830196F5CF80E047
:102CE00090E0883100E090073CF400E0FC01E55AF8
:102CF000FB4F00830196F5CF80E090E0803100E04B
:102D000090073CF400E2FC01E455FC4F008301967F
:102D1000F5CF80E090E0803100E090073CF400E0E7
:102D2000FC01EC56FB4F00830196F5CF822F912FCB
:102D30000895ECEBF3E000810E7F0083ECEBF3E011
:102D400000810D7F0083ECEBF3E001810B7F0183B9
:102D5000ECEBF3E00081077F0083ECEBF3E0008114
:102D60000F7E0083ECEBF3E000810F7D0083ECEB42
:102D7000F3E000810F7B0083ECEBF3E000810F7741
:102D80000083ECEBF3E001810E7F0183ECEBF3E0D9
:102D900001810D7F0183ECEBF3E000811181228141
:102DA00033810F7F1F7F2F7F307000831183228339
:102DB00033830895F8940E944B0F0E943E0F10E059
:102DC00002E00E94F3190E944C1A78940E94FC19A8
:102DD000B0DF35DF02E30093C103A8950E94031A18
:102DE0000023A1F5EDE1F7E0008100FF28C00E947B
:102DF000800FE2EDF0E00C94AB1EF8DA1EC01FDB92
:102E00001CC088DB1AC0E6DB18C025DC16C005DD57
:102E100014C06DDD12C012DE10C068DE0EC00E944C
:102E2000FD0F0BC00E94A11008C00E94331105C005
:102E30006DDC03C0B6DC01C047DB0E94FC19EDE18C
:102E4000F7E0008102FF02C00E94FC190091C1035B
:102E5000E0E0F1E00C94AB1E0091C203E8E3F1E086
:102E60000C94AB1E0E94F703B8CF0E940804B5CFA4
:102E70000E947304B2CF0E948A04AFCF0E94B804AC
:102E8000ACCF0E94C904A9CF0E943005A6CF0E94F2
:102E90004105A3CF0E945005A0CF0E945E059DCFA3
:102EA0000E946D059ACF0E94810597CF0E94B705B9
:102EB00094CF0E94C60591CF0E94D7058ECF0E9465
:102EC000DB058BCF0E94EC0588CF0E94610685CF81
:102ED0000E946F0682CF0E9486067FCF0E949306D3
:102EE0007CCF0E94A10679CF0E94E50676CF0E9492
:102EF000ED0673CF0E94030770CF0E946D076DCF60
:102F00000E947E076ACF0E94810767CF0E949207C6
:102F100064CF0E94960761CF0E94A7075ECF0E94F0
:102F200011085BCF0E943D0858CF0E94CE0855CFB4
:102F30000E944D0952CF0E9473084FCF0E94820811
:102F40004CCF0E948E0849CF0E949F0846CF0E9416
:102F5000510943CF0E94730940CF00E010E0009375
:102F6000C8031093C9030E94150A37CF0E94150A9F
:102F700034CF0E946D0A31CF0E94930B2ECF0E9456
:102F8000B80B2BCF0E94620928CF0E94FC0B25CFE3
:102F90000E940E0C22CF0E941E0C1FCF0E94470CD5
:102FA0001CCF0E94550C19CF0E946E0C16CF0E94A8
:102FB0007B0C13CF0E94BB0C10CF0E94C90C0DCF0D
:102FC0000E94D60C0ACF0E94DA0C07CF0E94E40CB4
:102FD00004CF0E94770D01CF0E94B50DFECE0E9456
:102FE000250CFBCE0E94370CF8CE0E94780EF5CE51
:102FF0000E948A0EF2CEE7E2F7E0008100610083D2
:103000000E944C1A0091C5031091C60300932D072E
:1030100010932E0700E814E00093290710932A0765
:1030200001E00E94B11A00917F040093C600ECEB0E
:10303000F3E001810B7F01830DE00093C103CDCE4E
:10304000E7E2F7E0008101FFC8CEE7E2F7E00081A8
:103050000061008300E00E94B11AE7E2F7E000811E
:103060000E7F00830FE714E00093290710932A07CF
:103070000091290710912A0700932B0710932C0722
:1030800003E00093C10301E00E94871A00EB14E003
:103090000E94C91B0E94DA1BA0CEE7E2F7E0008184
:1030A0000860008324EA33E004EF14E00E94461C29
:1030B000002339F400EB14E000931B0710931C0766
:1030C00006C000E117E200931B0710931C07E7E21C
:1030D000F7E000810F7E00830E944C1A0091C50327
:1030E0001091C60300932D0710932E0705EF14E0EF
:1030F0000093290710932A0701E00E94B11A00915A
:10310000F4040093C600ECEBF3E001810B7F018334
:1031100002E00093C10361CEE7E2F7E0008101FF26
:103120005CCE00E00E94B11AE7E2F7E000810E7F7A
:10313000008304EF14E00093290710932A070091FD
:10314000290710912A0700932B0710932C07E7E219
:10315000F7E0008103FF09C0ECEBF3E001810460BC
:10316000018300E00093C10338CE03E00093C10364
:1031700001E00E94871A00911B0710911C070E9412
:10318000C91B0E94DA1B29CE009127070570002376
:1031900021F1E7E2F7E00081077F008300E00E9471
:1031A000181A00E00E94871AE7E2F7E000810F7E1C
:1031B000008300911A07013029F4ECEBF3E0008161
:1031C0000061008300E000931A07ECEBF3E001815B
:1031D0000460018300E00093C103FFCD00E0009391
:1031E000C10301E00093C203ECEBF3E000810F7E2A
:1031F0000083F3CD00E00093C1030AE10093C20312
:10320000ECEBF3E000810F7E0083E7CD00E000935C
:10321000C10300E20093C203ECEBF3E000810F7EF8
:103220000083DBCD00E00093C10302E20093C20300
:10323000ECEBF3E000810F7E0083CFCD00E0009344
:10324000C10304E20093C203ECEBF3E000810F7EC4
:103250000083C3CD00E00093C1030AE20093C203E0
:10326000ECEBF3E000810F7E0083B7CD00E000932C
:10327000C10304E60093C203B0CD00E00093C10394
:1032800000E70093C203A9CD00E00093C10302E769
:103290000093C203A2CD00E00093C10303E70093B3
:1032A000C2039BCD8A93FA93EA933A922A921A9296
:1032B0000A927A936A935A934A933A932A931A9367
:1032C0000A938FB70091B900E2E0F2E00C94AB1ED4
:1032D00000E010E0009323071093240700E010E0C3
:1032E00000931F071093200705EC0093BC006AC0F1
:1032F0000091BB002091230730912407F901EC5580
:10330000FB4F0083E3E2F7E0008111810F5F1F4F65
:1033100000831183EFE1F7E0008111810F5F1F4F00
:103320000083118305EC0093BC004CC0EDE1F7E095
:1033300000810160008304E00093BC0043C000E012
:1033400010E00093250710932607009125071091A0
:103350002607F801EC55FB4F00810093BB00E5E226
:10336000F7E0008111810F5F1F4F0083118305EC8F
:103370000093BC0027C00091250710912607F80193
:10338000EC55FB4F00810093BB00E5E2F7E00081C4
:1033900011810F5F1F4F0083118305EC0093BC0068
:1033A00011C0EDE1F7E000810260008304E00093CA
:1033B000BC0008C0EDE1F7E000810460008304E98F
:1033C0000093BC008FBF09911991299139914991BE
:1033D0005991699179910990199029903990E991C1
:1033E000F99189911895202F220F212B2093BA0053
:1033F00024E02093BC00089500E000931D0705EC35
:103400000093BC0008951091BC00012F0170089535
:1034100002E00093B00000E00093B10000E00093F0
:10342000B2000AE00093B30000E00093700008953A
:10343000002369F010E01093B2001AE01093B3007B
:1034400012E01093700017E01093B100089510E09F
:103450001093700010E01093B100089502E004BDD5
:1034600000E005BD00E006BD01E107BD00E00093FE
:103470006E000895002351F010E016BD11E117BD54
:1034800012E010936E0013E015BD089510E0109344
:103490006E0010E015BD089508E10093C10006E03C
:1034A0000093C20007E410E01093C5000093C4002D
:1034B000D5DF00E0DFDFE7E2F7E0008104FF0DC0C9
:1034C0000FE714E00093290710932A070FE714E091
:1034D00000932B0710932C070CC004EF14E000930B
:1034E000290710932A0704EF14E000932B07109389
:1034F0002C07E7E2F7E000810D7F0083E7E2F7E0C9
:1035000000810E7F008300E000932F0708950E9442
:10351000F51EA02FAA23D9F0E7E2F7E0008104FD11
:103520000DC080E090E0863202E090073CF400E0BD
:10353000FC01EC50FB4F00830196F5CF8FDF01E0DB
:1035400099DF0091C10000680093C10007C000919D
:10355000C1000F770093C10000E08CDFE3E00C9422
:10356000FE1E002331F01091C10010641093C100C1
:1035700008951091C1001F7B1093C1000895FA9324
:10358000EA934A933A932A931A930A934FB7E7E23E
:10359000F7E0008104FF19C00091C600E0912907FF
:1035A000F0912A0700832091290730912A0700E92A
:1035B00014E02017310709F1E9E2F7E000811181F9
:1035C0000F5F1F4F0083118318C00091C600E09168
:1035D0002907F0912A0700832091290730912A07B3
:1035E00009E117E02017310741F0E9E2F7E0008137
:1035F00011810F5F1F4F008311834FBF09911991F4
:10360000299139914991E991F9911895FA93EA93A1
:103610002A931A930A932FB700912D0710912E0722
:10362000012B41F0EDE2F7E00081118101501040E3
:103630000083118300912D0710912E07012B81F03B
:10364000E0912907F0912A0700810093C600E9E282
:10365000F7E0008111810F5F1F4F0083118305C0C8
:10366000E7E2F7E00081026000832FBF0991199122
:103670002991E991F99118958A93FA93EA933A92EC
:103680002A921A920A927A936A935A934A933A9395
:103690002A931A930A938FB7E7E2F7E0008104FFB9
:1036A00035C000912F07039500932F0700912F0736
:1036B0000A3009F05DC000E000932F0700912B074E
:1036C00010912C072091290730912A070217130720
:1036D00009F04EC02091290730912A070FE714E026
:1036E000201B310B51F0E7E2F7E00081016000831D
:1036F00000E0C0DE00E00BDF3BC000912907109125
:103700002A0700932B0710932C0732C000912F0734
:10371000039500932F0700912F070A3049F500E029
:1037200000932F0700912B0710912C072091290758
:1037300030912A0702171307D9F4209129073091F5
:103740002A0704EF14E0201B310B51F0E7E2F7E009
:1037500000810160008300E08DDE00E0D8DE08C05B
:103760000091290710912A0700932B0710932C072B
:103770008FBF099119912991399149915991699175
:1037800079910990199029903990E991F99189914D
:1037900018959A938A93C801E7E2F7E000810B7FBE
:1037A0000083809332079093330700E041DE8991D4
:1037B00099910895E8E2F7E000810260008328DE35
:1037C00001E036DE08958A93FA93EA933A922A92B8
:1037D0001A920A927A936A935A934A933A932A9343
:1037E0001A930A938FB7E8E2F7E0008101FD15C054
:1037F000E0E3F7E000811181015010400083118364
:103800000091300710913107012B39F400E010DEF0
:10381000E8E2F7E000810E7F0083E8E2F7E0008154
:1038200001FF15C0E2E3F7E0008111810150104073
:10383000008311830091320710913307012B39F473
:1038400000E0F6DDE7E2F7E00081046000838FBF6F
:1038500009911991299139914991599169917991D8
:103860000990199029903990E991F99189911895C9
:10387000009330071093310708959A938A93C801F3
:103880008C010E944D1F8991999108950E94F41E08
:10389000D801C9019C018D010E94571F012B11F015
:1038A00001E001C000E0E4E00C94FD1E0E94F11E66
:1038B000C801D9016C908C01E0DF28018D01DDDFAA
:1038C000980100E010E00415150558F5FC01E00F23
:1038D000F11F5081561511F5B201601B710B621773
:1038E0007307E0F041E060E070E06217730790F466
:1038F0000B01000E111EFC01E00DF11D5081FD01B8
:10390000E60FF71F0080501511F040E003C06F5F15
:103910007F4FEBCF413011F4020F04C00F5F1F4FF8
:10392000D2CF00E0E7E00C94FA1E0E94F41ED8010A
:10393000C9019C018D010E94421FE4E00C94FD1E10
:103940000E94F41ED801C9019C018D010E94301F04
:10395000E4E00C94FD1E0E94F01ED80180E02D01D1
:1039600000E010E0063020E0120740F420E0F8010B
:10397000EC5CF84F20830F5F1F4FF4CF80E00A2FDD
:103980000B2B41F083954AE050E08D010E948E1E82
:10399000D801F5CF882321F400E3009334071CC03D
:1039A000682E772401E0601600E07006ACF04AE073
:1039B00050E082010E948E1E405DF301ED5CF84FE5
:1039C00040834AE050E082010E948E1E28010FEFE2
:1039D000600E0FEF701EE6CFE8E00C94F91E0E9417
:1039E000F41E642F652BE1F0B801621B730B0B0111
:1039F000B801640F751F61507040DB0180E090E0FA
:103A0000841795076CF4B001719561957040FD01C4
:103A1000E60FF71F6081FD01608311970196F0CFDB
:103A2000E4E00C94FD1E0E94F01EC801622E2224C8
:103A3000332420E030E060E070E00024112477249B
:103A400006141704ACF4FC0100810C3259F4022F67
:103A5000032B31F490018C010F5F1F4F280102C02E
:103A6000B00106C0019601E0000E00E0101EE7CF95
:103A7000022F032B19F0062F072B19F400E010E09A
:103A800059C0162F022F101B1A95B12FBB2311F00E
:103A9000B63018F000E010E04DC010E01B1788F4BD
:103AA000F2010081003338F4F20100810A3318F08A
:103AB00000E010E03FC001E0400E00E0501E139512
:103AC000EDCF0B2F10E0119501951040400E511EC7
:103AD000AB2FAA2371F1A13041F4F201008110E073
:103AE00000531040200E311E1EC041E050E0E0E0C7
:103AF000F0E00A2F10E001501040E017F10754F4F5
:103B00000AE0002E11248A01A0010E94861EA8014D
:103B10003196EFCFF201008110E0005310400E9477
:103B2000861E200E311E01E0400E00E0501EAA95B8
:103B3000D0CF8101E8E00C94F91E0E94F21EA8018A
:103B40000024112460E070E080E090E0222444240E
:103B5000552489010150104040165106A8F4FA017D
:103B6000E40DF51D00810D3051F4FA01E40DF51D51
:103B700001810A3021F4042D0E5F202E05C001E0E2
:103B8000400E00E0501EE5CF422C55248901015023
:103B9000104040165106D8F4FA01E40DF51D0081DD
:103BA0000D3081F4FA01E40DF51D01810A3051F464
:103BB00002E0400E00E0501EB2018A01060F171FFE
:103BC000D80105C001E0400E00E0501EDFCF2B0100
:103BD0008901015010404016510698F4FA01E40D95
:103BE000F51D00810D3041F4FA01E40DF51D018150
:103BF0000A3011F4C20105C001E0400E00E0501E81
:103C0000E7CF062F072B19F0082F092B19F400E036
:103C100010E02CC0FD0100810A3261F4FD01018138
:103C2000083041F4FD010281013421F4FD010381DA
:103C30000A3019F000E010E019C01496FD0100816F
:103C4000013821F4FD010181023A19F000E010E091
:103C50000DC0129612965096FD0151804424FD012C
:103C6000008110E0400E511E02018001E6E00C943C
:103C7000FB1E0C01B80140E000E010E080E090E0A5
:103C8000F90131978E179F07A0F4FB01E80FF91F88
:103C900050815D3061F4FB01E80FF91F51815A300A
:103CA00031F44395423019F402968C0102C001961A
:103CB000E7CFC0010895192F282F80E090E08F30C2
:103CC00000E0900754F4FC01E653FC4F0081002310
:103CD00011F001E003C00196F2CF00E0822F912F96
:103CE000089500008895FECF0FE30DBF01E00EBFE1
:103CF000C0E2D1E00E94061F002311F00E94161FAF
:103D00000E94DA160E94711E0C94711E149F102DD1
:103D1000059F100D049F002D110D089500241124FE
:103D2000EFE0001F111F001C111C0416150610F0F7
:103D3000041A150AEA95AAF7001F111FA0010095A1
:103D4000109508957591659155914591159011FAC9
:103D5000259035900895F9DF041B10E003C0F4DFCF
:103D6000041B150B20E030E005C0ECDF041B150B35
:103D7000260B370BB8F010FC17C045910590E00FEB
:103D8000F11F0417100540E02407340758F436F4F7
:103D900004910024F101E01BF0090994E00FF11FE8
:103DA00025903590F101099411F4D6F7F1CF3196B1
:103DB0000EF0319650E060E070E045914B3F48F0E6
:103DC00089F34F3F29F04E3F11F075916591559160
:103DD0004591041B150B260B370B39F318F3E7CF6E
:103DE0007A926A925A924A92BA93AA939A938A932F
:103DF00008957F806E805D804C80BB81AA8199810F
:103E00008881F0E0EC0FFD1FEF01089501E00895B7
:103E100020E006D0E9F70895259102D0E9F708954A
:103E20002D9301501040202F212B089588EF9EE301
:103E3000FC0105911491FC013296A591B491FC010D
:103E4000349625913491422F432B19F0F901E4DF88
:103E500001C0DEDF06961FE38430910748F3089522
:103E6000A80102C00F5F1F4FF80160816623D1F7E0
:103E7000F90161919F01F80161938F016623C1F7F8
:103E80008A010895A801F90161919F01F8016193E8
:103E90008F016623C1F78A010895F80101C03196A8
:103EA00020812223E1F7E01BF10B8F0108950E948E
:103EB000F41EF9014081442319F41BC00F5F1F4F0A
:103EC000F8014081442399F080E090E001C0019620
:103ED000D901A80FB91FF801E80FF91F40815C91C3
:103EE000451761F7FD014181442389F702C000E0D5
:103EF00010E0E4E00C94FD1E7C024001043F7E03D0
:103F0000BC03000041542B43495053544154555372
:103F10000D00004F4B0053544154453A20434F4E3F
:103F20004E454354204F4B0053544154453A204989
:103F30005020494E495449414C0053544154453A4C
:103F40002049502053544152540053544154453A4F
:103F500020495020434F4E46494700535441544551
:103F60003A20495020475052534143540053544142
:103F700054453A204950205354415455530053540A
:103F80004154453A2054435020434F4E4E454354EC
:103F9000494E470053544154453A2054435020431E
:103FA0004C4F53494E470053544154453A205443D3
:103FB0005020434C4F5345440053544154453A20FC
:103FC0005044502044454143540041542B434950F0
:103FD000534855540D000053485554204F4B004151
:103FE000542B4349504D55583D300D000041542B42
:103FF00043494943520D000041542B434946535213
:104000000D00002B43444E5347495000434F4E4E42
:10401000454354004641494C0041542B43495043C9
:104020004C4F53453D300D000053544154453A2008
:10403000495020434F4E4E454354204F4B0041546E
:104040002B43495053454E443D00000D00002B4387
:104050004D45204552524F520053454E4420464153
:10406000494C0053454E44204F4B003E0041542BD9
:1040700043495052584745543D322C33300D0000CF
:104080002B43495052584745543A20322C00455250
:10409000524F520041542B43495052584745543DCA
:1040A000322C000041542B43495052584745543D4F
:1040B000310D000041545A0D000041540D000041E3
:1040C000542B4950523D393630300D0041542B4964
:1040D00043463D332C330D0041542B4946433D307C
:1040E0002C300D00415451300D00415456310D001B
:1040F000415445300D0041542B434D45453D310D54
:104100000041542B43495052584745543D310D000E
:1041100041542B474D520D00494E495449414C00E2
:10412000535441525400434F4E4649470047505262
:10413000534143540053544154555300434F4E4E42
:10414000454354494E4700434C4F53494E47004363
:104150004C4F534544004445414354004F4B00529B
:1041600065766973696F6E0041542B435553440063
:10417000200000000000000000000000000000001F
:00000001FF
:00000001FF
